:1000000000308A00CE2900000A108A100A118207E7
:1000100028340C34013406340A108A100A1182077D
:10002000413468346F346A3400341B308400000873
:100030000319292801308D008C018C0B1D288D0B94
:100040001C284A308C008C0B232800000000800BF9
:100050001A2800340608C339A200210D8C008C0D2B
:10006000FC308C050C083C392204860006148316EB
:100070000610000083120610831606108312003447
:100080009F08031D4528861046288614831686106F
:100090008312A00E2008A1002A20A00E2008A10093
:1000A0002A200D308C008C0B5328003414309B0018
:1000B0001520C3308316860583128610831686109A
:1000C0008312061083160610831298011808023C4A
:1000D000031C722802309B0015200330A1002A2047
:1000E000980A66280D308C008C0B74280230A10011
:1000F0002A200D308C008C0B7B2898011808023CBC
:10010000031C8E281808042099009F011908A000DC
:10011000402002309B001520980A7E28D229013009
:100120001B029D001C08023C031D982840309D07BF
:100130001D0880389E009F011E08A000402000344A
:100140001A088C000C300C020319B3280A300C0278
:100150000319BB280D300C020319C12808300C020A
:100160000319C628CB289F010130A000402002308F
:100170009B001520D72801309B0002309C008F2067
:10018000D72801309B009C008F20D7289F0110307A
:10019000A0004020D7281A081F3C031CD128073094
:1001A0009A0501309F001A08A0004020D72800348B
:1001B0001D088400800104309E009E080319EE286B
:1001C000831685158312851DE72804309E0029308B
:1001D0008C008C0BE92800009E03DD288316851512
:1001E0008312851DEE28DD308C008C0BF528000075
:1001F00000001C08840083168515003083128519C1
:10020000013080009E011E08033C031C2829A630F3
:100210008C008C0B092900001D0884000310000CC1
:100220008C008000831685158312851D1C291D08EE
:1002300084000830000780001F182029051121299B
:10024000051583160511013083129F069E0A0329A6
:1002500000308D0000341A309C0019089D00D82011
:100260008D080319362901308D0086299A08031D4F
:100270002B291908840000080F3C03194229023079
:100280008D0086291A309C0018089D00D8208D0802
:1002900003194D2901308D0086299A08031D532921
:1002A00003308D0086291A309C0019089D00D82043
:1002B0008D0803195E2901308D0086299A08031DD7
:1002C000642903308D0086291A309C001B309D0064
:1002D000D8208D0803196F2901308D0086299A08CE
:1002E000031D752903308D00862918088400000835
:1002F0009C001908840000081C070F391B02031911
:10030000842903308D00862900308D00FA291B08CE
:100310008D011A0203188F291A088C009B298C0161
:1003200008309C009A0D8C0D1B080C0203188C00E1
:100330008D0D9C0B922900340D0818089A0064302A
:100340009B0087210C0898000D083030031DAF2951
:10035000191899159919B529191A2030B129991127
:1003600019128D070D089A00A02018089A000A306B
:100370009B0087210C0898000D083030031DC4290C
:100380009919C829191A20308D070D089A00A02044
:100390003030980718089A00A020003484011F30DC
:1003A0008305562805309B001520980118080C205D
:1003B000980A9A00A02004301802031DD6290330A1
:1003C00099002E309A00A020990BE1290230980064
:1003D00096309B001520980BE8298E018F01900123
:1003E0009101920193019401950116309800173004
:1003F00099002B298D080319FF29920AA62A01309A
:100400001602FD3E0318102A033EA82A17088E0084
:10041000900A102A17088F00910A102A950A102AAC
:1004200001309B009C008F2058309A00A0200E08BD
:100430009800113099009C2120309A00A0201008CB
:100440009800103099009C211208980010309900F3
:100450009C2113089800103099009C2120309A00AC
:10046000A02020309A00A02001309B0002309C0088
:100470008F2059309A00A0200F0898001130990061
:100480009C2120309A00A02011089800103099007B
:100490009C2114089800103099009C2115089800A0
:1004A000103099009C2120309A00A02020309A0022
:1004B000A020831605108312051401309B0015201F
:1004C0000E08970017089703003A0319712A153090
:1004D0008C008C0B692A00009708031D702A0030DD
:1004E000622A831605108312051083168510831265
:1004F000851401309B0015200F08970017089703FB
:10050000003A03198D2A15308C008C0B852A0000C7
:100510009708031D8C2A00307E2A831685108312CB
:1005200085100E081E3C8D000F080D02970017085D
:100530009703003A0319A62A15308C008C0B9E2ACB
:1005400000009708031DA52A0030972AF5296300AB
:0E0550000A108A140A118207062A0A2A0E2AA5
:02400E00F13F80
:00000001FF
